:101100003140000AB240805A20013F4000000F9356
:1011100005242F839F4F78130002FB233F400400D8
:101120000F9304241F83CF430002FC2330400C1391
:1011300030403411001392D30202B1C0F00000001D
:101140000013829300020324E2C235000013E2D2AE
:1011500035000013A2931E0101240013E2D23500D2
:10116000FC3F0F1282430002E2C30200E2B302001E
:10117000F9233F4100130E430E9F132C03430343F7
:10118000034303430343034303430343034303432F
:101190000343034303430343034303431E530E9F8D
:1011A000ED2B3041B240805A2001C2432100C2439E
:1011B0002900C2431900C2431D00C2433100E2426C
:1011C0003500C2432600C2432E00C2431B00C24367
:1011D0001F00C2433300C2433700D2432200C24340
:1011E0002A00C2431A00F240FCFF1E00F2403F00FA
:1011F0003200E2423600C2432400C2432C00C24304
:101200002500C2432D00F2F0DFFF5400E2C30200CC
:10121000E2B30200FB23E2425400B2400401600149
:10122000B24000807201B24010006201824364014A
:1012300082436601B2D01000600182430002B240D6
:1012400004028001B240D8049201B240E50094014A
:10125000B24010008201B240D0008401B2D0100030
:101260008001E2D300003041F2F0C0FF3100F2F023
:1012700003001D0030418F113F9003003D242F9249
:1012800017341F930D242F93012430415E930424BF
:10129000F2D080FF1D003041F2D040001D003041EF
:1012A0005E930324E2D331003041D2D33100304188
:1012B0003F90050019243F9005000E383F9006002E
:1012C000012430415E930424F2D0100031003041FB
:1012D000F2D02000310030415E930324E2D21D00A1
:1012E0003041F2D21D0030415E930324E2D231003E
:1012F0003041F2D2310030415E930424F2D020001C
:101300001D003041F2D010001D0030413140000A74
:101310002A42B012A41132D2D2D321003F400F0092
:10132000B0127611D2C32100B24066067201824328
:1013300000023A90060001381A43B01268121B43AB
:101340000B9A14244E434F4BB01276121B533B9012
:101350000600F63B3F405F00B0127611B0126812F3
:10136000924300021A5332D01000E13F5E434F4ACD
:08137000EB3F30407613FF3F14
:10FFE0003011301130113011301130113611301103
:10FFF00030113011301130115411421162110011C1
:0400000300001100E8
:00000001FF
